:10000000830100308A001D288C00030883019B00B7
:100010008E0A03198F0A3A300F02993003190E0223
:10002000031C14288D018D0A0B118330831281006B
:100030001B0883008C0E0C0E09000D3084001B3051
:1000400026208301842B04068001840A04060319F8
:04005000003423282D
:1006EE0098000430990053309A009A0B7C2B990B8A
:1006FE007A2B980B782B831208001F3083168600F6
:10070E0001308500831286018501831681128111C5
:10071E000110811401118B178B120B119201FA30FB
:10072E0083127723920A04301202031C962B900137
:10073E008E018F010518A12B900A33301002031C75
:10074E00FD2B851492018D018330831281008B164F
:10075E00061AB62B0D03031DAF2B85109E2B8B1285
:10076E008E018F011208133E840006080F39800097
:10077E00061ABF2B920A05301202031CAA2B130B6A
:10078E00A92B1408023A031DA92B1508033A031DC1
:10079E00A92B1608043A031DA92B17080B3A031DA3
:1007AE00A92B83120515061EDA2B06080F399100A8
:1007BE00110BE22B86161108023A031906171108BF
:1007CE00033A031986171108043A03198612110801
:1007DE00053A031906131108063A03198613110870
:1007EE000C3A031DDA2B851005119E2B0518A12B33
:0207FE00FD2BD1
:02400E00F1FFC0
:00000001FF
